:020000040000FA
:0400000057EF03F0C3
:040008001BEF08F0F2
:0800180064EF08F00F0B176EF6
:10002000000EF76E3A0EF66E1750F626D8B0F72A85
:10003000F29E0800F28EF550120030313233343522
:1000400036373839414243444546000EF86E150EA6
:10005000F76E3E0EF66E2DEC0AF01EC039F029D078
:10006000000EF86E150EF76E440EF66E2DEC0AF0CB
:1000700025C039F01ED0000EF86E150EF76E4A0E30
:10008000F66E2DEC0AF026C039F013D0000EF86E93
:10009000150EF76E500EF66E2DEC0AF008EC0BF014
:1000A000D8901F30396E6AEC15F0020E586E3BEF97
:1000B00014F058EC0DF0F4EC0EF083EC15F0030E98
:1000C000586E596A5B9467EF14F00FB26AD0000E55
:1000D00022EC0AF04BC14EF04CC14FF04DC150F034
:1000E0004EC151F04FC152F083EC15F0080E586E1E
:1000F000596A5C8667EC14F011BA22D00FA00DD0BB
:10010000000EF86E150EF76E320EF66E2DEC0AF03C
:1001100008EC0BF01CC039F00CD0000EF86E150E78
:10012000F76E380EF66E2DEC0AF008EC0BF01DC0E1
:1001300039F06AEC15F0030E586E3BEC14F008D061
:10014000000EF86E150EF76E2A0EF66E2DEC0AF004
:1001500099EC05F012E25F6603D025EC00F00CD0BC
:10016000010E5F6203D030EC00F006D0020E5F6239
:1001700003D03BEC00F000D011D05F6603D046EC1A
:1001800000F00CD0010E5F6203D030EC00F006D01E
:10019000020E5F6203D025EC00F000D03FD8E9D812
:1001A0003BD0000E22EC0AF04BC14EF04CC14FF098
:1001B0004DC150F04EC151F04FC152F083EC15F0DB
:1001C000080E586E596A5C8667EC14F011BA13D0A9
:1001D000000EF86E150EF76E380EF66E2DEC0AF066
:1001E00008EC0BF01DC039F06AEC15F0030E586EE8
:1001F0003BEC14F008D0000EF86E150EF76E2A0EC8
:10020000F66E2DEC0AF0B5D8000EF86E140EF76EEF
:10021000F40EF66E2DEC0AF087D8120027C039F0E4
:10022000396608D0000EF86E140EF76EAC0EF66E3E
:100230002DEC0AF0010E396208D0000EF86E140E93
:10024000F76EB20EF66E2DEC0AF0020E396208D08F
:10025000000EF86E140EF76EB80EF66E2DEC0AF066
:10026000030E396208D0000EF86E140EF76EBE0E43
:10027000F66E2DEC0AF0040E396208D0000EF86E0E
:10028000140EF76EC40EF66E2DEC0AF0050E3962F0
:1002900008D0000EF86E140EF76ECA0EF66E2DEC36
:1002A0000AF0060E396208D0000EF86E140EF76ED2
:1002B000D00EF66E2DEC0AF0070E396208D0000E53
:1002C000F86E140EF76ED60EF66E2DEC0AF0080ED0
:1002D000396208D0000EF86E140EF76EDC0EF66E62
:1002E0002DEC0AF0090E396208D0000EF86E140EDB
:1002F000F76EE20EF66E2DEC0AF00A0E396208D0A7
:10030000000EF86E140EF76EE80EF66E2DEC0AF085
:100310000B0E396208D0000EF86E140EF76EEE0E5A
:10032000F66E2DEC0AF01200236602D0090E1ED0E4
:10033000010E236202D0080E19D0020E236202D0F1
:10034000070E14D0030E236202D0070E0FD0040E46
:10035000236202D0050E0AD0050E236202D0050EDC
:1003600005D0060E236202D0040E00D022EC0AF063
:100370001200236608D0000EF86E150EF76E560EAA
:10038000F66E2DEC0AF0010E236208D0000EF86E16
:10039000150EF76E5C0EF66E2DEC0AF0020E23625F
:1003A00008D0000EF86E150EF76E620EF66E2DEC8C
:1003B0000AF0030E236208D0000EF86E150EF76ED9
:1003C000680EF66E2DEC0AF0040E236208D0000EC3
:1003D000F86E150EF76E6E0EF66E2DEC0AF0050E29
:1003E000236208D0000EF86E150EF76E740EF66ECE
:1003F0002DEC0AF0060E236208D0000EF86E150EE2
:10040000F76E7A0EF66E2DEC0AF012005A0E74ECAE
:1004100009F05A0E74EF09F0F9DF410E74EC09F09F
:10042000550E74EC09F024C039F058EC0DF0F4ECE2
:100430000EF083EC15F0020E586E596A5B885C84EE
:100440005B9467EC14F027D1E1DF410E74EC09F006
:10045000440E74EC09F0E7D7460E74EC09F0410E37
:1004600074EC09F0310E74EC09F0300E74EC09F004
:10047000340E74EC09F04BC14EF04CC14FF04DC13D
:1004800050F04EC151F04FC152F083EC15F0080E00
:10049000586E596A5B885C8467EC14F0FCD0B6DF58
:1004A000460E74EC09F0410E74EC09F0300E74EC59
:1004B00009F0300E74EC09F04BC14EF04CC14FF016
:1004C0004DC150F04EC151F04FC152F083EC15F0C8
:1004D000090E586E596A5B885C8467EC14F0DBD0B7
:1004E00095DF410E74EC09F0520E74EC09F01EC059
:1004F00039F058EC0DF0F4EC0EF083EC15F0030E2F
:10050000586E596A5B885C845B8467EC14F0C3D0D6
:100510004D0E74EC09F0550E74EC09F0300E11AA72
:10052000310E74EC09F0B7D071DF4D0E74EC09F0A8
:10053000410E74EC09F0300E11BA310E74EC09F072
:10054000AAD064DF540E74EC09F04F0E74EC09F07D
:1005500008EC0BF026C039F037D058DF500E74ECA1
:1005600009F0430E74EC09F008EC0BF025C039F0EB
:100570002BD04CDF4C0E74EC09F0410E74EC09F0FA
:1005800008EC0BF01DC039F01FD0410E74EC09F0DF
:10059000470E74EC09F008EC0BF01DC039F06AEC62
:1005A00015F0030E586E596A5B885C843BEC14F0BE
:1005B00072D02CDF410E74EC09F0470E74EC09F098
:1005C00008EC0BF01CC039F06AEC15F0030E586E05
:1005D000596A5B885C843BEC14F05DD017DF430EF6
:1005E00074EC09F0530E74EC09F008EC0BF0D890A1
:1005F0001F30396E6AEC15F0020E586E596A5B882E
:100600005C843BEC14F047D001DF4D0E74EC09F034
:10061000410E74EC09F03FD0F9DE410E74EC09F0A4
:10062000520E74EC09F037D0F1DE470E74EC09F08D
:10063000410E74EC09F02FD0E9DE4C0E74EC09F099
:10064000410E74EC09F027D0E1DE410E74EC09F0A4
:10065000470E74EC09F01FD0D9DE490E74EC09F096
:10066000460E74EC09F017D0D1DE500E74EC09F090
:10067000430E74EC09F00FD0C9DE540E74EC09F08F
:100680004F0E74EC09F007D0C1DE430E74EC09F094
:10069000530E74EC09F03B0E74EF09F06F6B13EE20
:1006A00000F0320E0A6EE66A0A2EFDD712006FECD9
:1006B00008F0EBEC08F00FEC09F0FDEC08F080EC32
:1006C00009F044EC09F04EEC03F0B8EC09F001013C
:1006D0004B6B4C6B4D6B4E6B4F6B00011082FF0EE2
:1006E000286EFF0E276E320E206E0FB20F9018523A
:1006F00025E018C039F058EC0DF0F4EC0EF0C9EC20
:1007000005F00AEC0FF04BC153F04CC154F04DC151
:1007100055F04EC156F04FC157F0CDEC0FF04EC022
:100720004BF14FC04CF150C04DF151C04EF152C091
:100730004FF122EC05F01082108E186A10A203D03F
:10074000109265EC00F019523BE00FB234D099ECF6
:1007500005F018E25F6605D019C039F064EC05F0C9
:1007600010D0010E5F6205D019C039F070EC05F0B1
:1007700008D0020E5F6205D019C039F07CEC05F09C
:1007800000D017D05F6605D019C039F088EC05F0AD
:1007900010D0010E5F6205D019C039F070EC05F081
:1007A00008D0020E5F6205D019C039F064EC05F084
:1007B00000D0196A108219C039F070EC05F0196A7E
:1007C0001A5212E00FB20AD01AC039F00FA0BDECD5
:1007D00005F00FB0A5EC05F01A6A10821AC039F0C6
:1007E000B1EC05F01A6A108277EC07F053E391EC54
:1007F00007F0010E1B620ED02306FF0E236201D00C
:10080000236A4EEC07F03FEC05F01082108EF3ECFB
:1008100008F03ED0020E1B620FD0232A070E23627F
:1008200002D0060E236E4EEC07F03FEC05F010826E
:10083000108EF3EC08F02CD0030E1B6206D05F2A5A
:10084000030E5F6201D05F6A23D0040E1B6208D0E2
:10085000117A0FB288EC02F00FA294EC02F018D0DB
:100860000C0E1B6203D0D3EC07F012D00B0E1B62F0
:1008700006D00F7205EC09F0B4EC08F0FF000E0E84
:100880001B6206D00FB204D00F7005EC09F000D047
:100890001082186A10B410D05DEC09F00DE33B0E25
:1008A0006C6302D0108408D06C5113EE00F06F51CD
:1008B000E1266CC0E6FF6F2B10A444D010940FB259
:1008C00033D08CEC06F003E325EC07F010825CECEF
:1008D00006F003E3E7EC06F010824DEC06F003E3CC
:1008E000BFEC06F010823EEC06F003E3B5EC06F038
:1008F000108274EC06F003E39DEC06F010822FECFE
:1009000006F003E3DDEC06F0108217EC06F003E3DB
:10091000C9EC06F0108208EC06F003E3ACEC06F03C
:1009200010824EEC03F00ED06BEC06F003E3F1EC1A
:1009300006F0108283EC06F003E308EC07F0108267
:100940004EEC03F00FB205D010A803D01098B9EC0C
:1009500002F00FB206D010A609D01096D9EC02F022
:1009600005D010A603D01096C5EC02F00FB205D04A
:1009700010AA03D0109A70EC02F0206630D0320E2C
:10098000206E0FB21BD0226603D02CEC03F022D0D5
:10099000010E226209D024EC03F01CEC03F03CECC5
:1009A00003F004EC03F016D0020E2262FDD70CEC2B
:1009B00003F044EC03F034EC03F00CD0010E22629F
:1009C00003D025EC03F006D0020E226203D02DECFA
:1009D00003F000D0222A030E226201D0226A10AC5A
:1009E00004D0109C0FA2EEEC02F010AE09D0109EC5
:1009F0000FA24FEC02F00FB22CEC02F0320E206E80
:100A000011A004D011900FA224EC02F011A204D086
:100A100011920FA20CEC02F011A404D011940FA2B9
:100A2000ADEC02F011A604D011960FA2A1EC02F0D9
:100A30002850275CD8B404D05F6A27C028F0108201
:100A400077EF03F04BC14EF04CC14FF04DC150F069
:100A50004EC151F04FC152F09CD88AEC0FF08BEC94
:100A60000CF097D80AEC0FF04EC04BF14FC04CF190
:100A700050C04DF151C04EF152C04FF112004BC168
:100A80004EF04CC14FF04DC150F04EC151F04FC12E
:100A900052F07FD88AEC0FF0C7EC0CF07AD80AEC51
:100AA0000FF04EC04BF14FC04CF150C04DF151C052
:100AB0004EF152C04FF11200430E576EFA0E566EB1
:100AC000536A546A556A120039501E261EAE01D070
:100AD0001E6A780E1E6402D0780E1E6E108A1200F6
:100AE0003950252625AE01D0256A640E256402D032
:100AF000640E256E118412003950262626AE01D0D0
:100B0000256A640E266402D0640E266E11861200D9
:100B100039501F26120E1F6002D0120E1F6E500E8B
:100B20001F6402D0500E1F6E108C120028C039F0C6
:100B300002D027C039F0030E395C05E0040E395CA1
:100B400002E0D8901200D880120039501C261CAE4A
:100B500001D01C6A640E1C6402D0640E1C6E1086E8
:100B6000120039501D261DAE01D01D6A640E1D6491
:100B700002D0640E1D6E1086120039501D261DAE67
:100B800001D01D6A640E1D6402D0640E1D6E1088B3
:100B90001200236603D025EC11F023D0010E23624E
:100BA00003D034EC11F01DD0020E236203D007EC09
:100BB00011F017D0030E236203D03CEC11F011D0DA
:100BC000040E236203D05CEC05F00BD0050E23620B
:100BD00003D044EC11F005D0060E236202D04CEC99
:100BE00011F0120013EE00F0020E0A6E20EE64F017
:100BF000E6CFDEFF0A2E07D0120013EE00F0040E3F
:100C00000A6E20EE64F0E6CFDEFF0A2EFCD712005B
:100C1000F4DF5A0E64638FD05A0E65638CD04D0E8C
:100C2000666389D0410E676386D0D8801200E5DF05
:100C30005A0E646380D05A0E65637DD0540E66638D
:100C40007AD04F0E676377D0D8801200D6DF500E6F
:100C5000646371D0430E65636ED0D8801200CDDF1F
:100C60005A0E646368D05A0E656365D0500E666391
:100C700062D0430E67635FD0D8801200BEDF5A0E89
:100C8000646359D05A0E656356D0410E666353D0E3
:100C9000520E676350D0D8801200AFDF5A0E6463E3
:100CA0004AD05A0E656347D04C0E666344D0410E5D
:100CB000676341D0D8801200A0DF5A0E64633BD036
:100CC0005A0E656338D0410E666335D0470E6763B0
:100CD00032D0D880120086DF410E64632CD0470EDC
:100CE000656329D0D880120088DF5A0E646323D050
:100CF0005A0E656320D0430E66631DD0530E6763A2
:100D00001AD0D880120079DF490E646314D0460EE1
:100D1000656311D0D880120070DF5A0E64630BD067
:100D20005A0E656308D0490E666305D0460E6763A8
:100D300002D0D8801200D8901200FAEC0AF004C356
:100D400030F005C32FF03AEC16F05AEC0EF02FC03D
:100D50001FF0D8901F36120004C339F0310E3962EB
:100D600002D0118A01D0119A120013EE05F020EE84
:100D700031F0030E0A6E41D82FC01EF0120013EEA0
:100D800004F020EE31F0030E0A6E37D82FC01DF0AC
:100D9000120013EE04F020EE31F0030E0A6E2DD88F
:100DA0002FC026F0120013EE02F020EE31F0030EF9
:100DB0000A6E23D82FC025F0120013EE04F020EEA7
:100DC00031F0030E0A6E19D82FC025F0120013EE71
:100DD00004F020EE31F0030E0A6E0FD82FC01CF085
:100DE000120013EE02F020EE31F0030E0A6E05D869
:100DF0002F5202E02FC01DF01200FAEC0AF0E6CFED
:100E0000DDFF0A2EFCD73AEC16F05AEC0EF0120079
:100E100013EE05F020EE36F0080E0A6EFAEC0AF03A
:100E2000E6CFDDFF0A2EFCD73AEC16F010EC0EF000
:100E300090EC0DF049C04BF14AC04CF14BC04DF164
:100E40004CC04EF14DC04FF1120013EE05F020EEF4
:100E500038F00A0E0A6EFAEC0AF0E6CFDDFF0A2E31
:100E6000FCD73AEC16F010EC0EF090EC0DF049C007
:100E70004BF14AC04CF14BC04DF14CC04EF14DC04E
:100E80004FF1FAEC0AF01FC330F020C32FF03AEC18
:100E900016F05AEC0EF02FC027F01200236602D095
:100EA000246A24D0010E236203D0010E246E1ED0CA
:100EB000020E236203D0030E246E18D0030E2362A9
:100EC00003D0040E246E12D0040E236203D0060E4B
:100ED000246E0CD0050E236203D0070E246E06D0BC
:100EE000060E236203D00C0E246E00D01200D890A0
:100EF00082A8D88082A6D88081ACD88081AED880E4
:100F00001200F5DFFEE31200F2DFFEE21200000E37
:100F100082A8010E82A6020E81AC030E81AE040EE1
:100F20001200EFDFF4DF1B6EC4EC08F0F0DF1B5C97
:100F3000F9E10A0E0A6E77EC07F034E3BEEC08F034
:100F40000A2EF9D70A0E1B261FEC0AF00B0E1B62A5
:100F500009D0000EF86E140EF76EFA0EF66E2DEC38
:100F60000AF020D00C0E1B6209D0000EF86E150E90
:100F7000F76E120EF66E2DEC0AF014D00E0E1B62F8
:100F800009D0000EF86E150EF76E1E0EF66E2DECE3
:100F90000AF008D0000EF86E150EF76EA00EF66E71
:100FA0002DEC0AF0B1D716C050F1000EF86E150EF8
:100FB000F76E800EF66E2DEC0AF0000EF86E150E30
:100FC000F76E8C0EF66E2DEC0AF008EC0BF016C0E6
:100FD00039F06AEC15F0020E586E3BEC14F0185222
:100FE0000DE018BE160618AE162A3F0E166402D083
:100FF0003F0E166E186AF2EC09F0DFD777EC07F0B7
:10100000EEE391EC07F0020E1B620FD0E1EC08F06A
:10101000000EF86E150EF76E940EF66E2DEC0AF0BB
:10102000B4EC08F01FEC0AF002D050C116F01082A8
:101030001FEC0AF01200EACF04F0E9CF03F0F2A2AD
:1010400005D0F29281B6182A81A61806F0A005D024
:10105000F09081B8192A81A81906F0A20DD0F0925B
:10106000F178F1A805D081AA1A2A81BA1A0604D00B
:1010700081AA1A0681BA1A2A69C0EAFF68C0E9FF84
:101080009EAA0ED0AE50ABA204D0AE50AB98AB88A7
:10109000F7D7EE6EF10EE95C02E102EE00F0F0D758
:1010A000EACF69F0E9CF68F09EA009D09E90206653
:1010B000200621662106580ECE6E9E0ECF6E04C00D
:1010C000EAFF03C0E9FF1100006ED8CF01F0E0CFC6
:1010D00002F002C0E0FF005001C0D8FF10000F0175
:1010E000700ED36E000E9B6E806A896A000E386F98
:1010F000000E926E816A8A6A000E396FFF0E936E3F
:10110000826A8B6AD80E946E000E3A6F846A000E63
:10111000966E000EC16E000EC06E000ED06ED00E28
:10112000F26E000EF16E180EF06E010E9D6E000E46
:10113000A06E000ED56E330ECD6E000EBA6E000E90
:10114000B16E0001FF0E0A6E00EE00F0EE6A0A2E8C
:10115000FDD7580ECE6E9E0ECF6E1200B2EC08F088
:10116000B4EC08F0B4EC08F0BAEC08F0BAEC08F013
:10117000BAEC08F0FA0E10D0C80E0ED0640E0CD0E7
:10118000320E0AD01E0E08D00A0E06D0050E04D06C
:10119000020E02D0010E00D0096E2D0E076E060E53
:1011A000086E072EFED7082EFCD7092EF6D71200A0
:1011B000000000000000000000000000000000002F
:1011C0001200010E0A6E00EE16F0000E056E36ECEF
:1011D00009F0BEEF08F0010E0A6E00EE16F0000EE8
:1011E000056E3DEF09F0010E0A6E00EE23F0010ED0
:1011F000056E36EC09F0BEEF08F0010E0A6E00EE47
:101200000FF0020E056E3DEF09F0010E0A6E00EEC2
:101210000FF0020E056E36EC09F0BEEF08F0010E7D
:101220000A6E00EE23F0010E056E3DEF09F0A6B246
:10123000FED705C0A9FF06C0A8FFA69EA69CA6844F
:10124000F29EF2BEFDD7550EA76EAA0EA76EA6821D
:1012500010A0F28EA6941200A6B2FED705C0A9FF78
:10126000A69EA69CA680A8CF06F01200EECF06F0A0
:10127000DEDF052A0A2EFAD71200EEDF06C0EEFFE7
:10128000052A0A2EFAD7120012EE00F0E1CF6AF01A
:10129000E2CF6BF0E1CF68F0E2CF69F00FB204D09B
:1012A000190EAF6EAC9403D0100EAF6EAC84AB8849
:1012B000AC98AB8EAC8A9D8A12006AC0E1FF6BC00D
:1012C000E2FF6851E15C02E1D8901200E6506C6FD9
:1012D000F10EE15C02E112EE00F0E1CF6AF0E2CF44
:1012E0006BF06C51D88012009EA8FED7AD6E120034
:1012F000ABA402D0AE50FCD79EAAFED7AE501200CF
:10130000BEEC08F08988BEEC08F08980BEEC08F0DD
:101310008996BEEC08F03A0E02EC0AF0090E02ECD7
:101320000AF0060E02EC0AF01E0E02EC0AF0390E6C
:1013300002EC0AF01B0E02EC0AF06E0E02EC0AF050
:101340007A0E02EC0AF0570E02EC0AF0380E02ECAC
:101350000AF00E0E02EC0AF03A0E02EC0AF0090E48
:1013600002EC0AF03C0E02EC0AF03CD868D81200FD
:101370000FB209D0000EF86E150EF76EAC0EF66EB9
:101380002DEC0AF008D0000EF86E150EF76EB80EB0
:10139000F66E2DEC0AF0000EF86E150EF76EC40E08
:1013A000F66E2DEC0AF0000EF86E150EF76ED00EEC
:1013B000F66E2DEC0AF0B2EC08F0000EF86E150E89
:1013C000F76EDC0EF66E2DEC0AF0000EF86E150EC0
:1013D000F76EE80EF66E2DEC0AF0B2EC08F01FEC9A
:1013E0000AF012003D0E02EC0AF016500F0B7009C5
:1013F00009D81650E838030B540904D83C0E02EC07
:101400000AF012008996296E1F0E03D08996296E64
:101410005F0E08D829500F0B05D829380F0B02D8BA
:1014200089861200126E080E136E89981232D8A0A7
:10143000899AD8B0898A8988132EF7D71200010EAD
:10144000E1DF000E8009DED72A6E2A380EEC00F0AC
:10145000DDDF2A500EEC00F0D9D70900F550F2DF9D
:101460000900F55002E0D2DFFBD71200200ECED7E4
:10147000146E36EC0AF0142EFCD71200205461735F
:10148000746520312020200020546173746520325F
:101490002020200020546173746520332020200018
:1014A000205461737465203420202000474C53423F
:1014B0000000475553420000474453420000474351
:1014C000574C00004743575500004720464D000049
:1014D0004720414D000047444755000047535045C1
:1014E00000004744474C00004753414D000047442B
:1014F000524D00004753445200000050775344526D
:101500002F436F6E7300004D7574654F4E2F4F461D
:10151000460000536574757020212020200000567D
:101520006F6C2E77656368732E00204D7574654F60
:101530004E0020566D3A000020566F6C000040416E
:1015400067630000404472760000404474750000F8
:101550004057704D3A002731487A0000272031303B
:1015600000002720353000002731303000002735BB
:10157000303000002720316B00002731306B000035
:10158000003D3D53455455503D3D3D00204B6F6E51
:1015900074723A002047657370656963682E210094
:1015A000005461737465206C616E670000506F7742
:1015B000657253445220200000534452436F6E73AF
:1015C0006F6C6500204857312E30302020202000DD
:1015D000405357312E303920202020002031312E29
:1015E00030342E323032310040286329444C344AA2
:1015F000414C200013D806D8346A356A366A376AF7
:10160000386A12002F6A306A316A326A336A12000D
:10161000396A3A6A3B6A3C6A3D6A1200F9DF3E6AFF
:101620003F6A406A416A426A12004E6A4F6A506AD3
:10163000516A526A12000EC153F00FC154F010C12A
:1016400055F011C156F012C157F012000EC14EF004
:101650000FC14FF010C150F011C151F012C152F042
:10166000120053C04EF054C04FF055C050F056C059
:1016700051F057C052F012004EC053F04FC054F01A
:1016800050C055F051C056F052C057F012004EC035
:101690000EF14FC00FF150C010F151C011F152C006
:1016A00012F1120013C14EF014C14FF015C150F0E9
:1016B00016C151F017C152F0120013C153F014C1FA
:1016C00054F015C155F016C156F017C157F012006D
:1016D00018C14EF019C14FF01AC150F01BC151F0A2
:1016E0001CC152F0120018C153F019C154F01AC1B4
:1016F00055F01BC156F01CC157F012001DC14EF031
:101700001EC14FF01FC150F020C151F021C152F055
:1017100012001DC153F01EC154F01FC155F020C16D
:1017200056F021C157F0120022C14EF023C14FF0F4
:1017300024C150F025C151F026C152F0120022C13F
:1017400053F023C154F024C155F025C156F026C1F1
:1017500057F0120027C14EF028C14FF029C150F0B8
:101760002AC151F02BC152F0120027C153F028C1F9
:1017700054F029C155F02AC156F02BC157F0120080
:1017800053C013F154C014F155C015F156C016F1F1
:1017900057C017F112004EC013F14FC014F150C0E2
:1017A00015F151C016F152C017F112004EC018F1D8
:1017B0004FC019F150C01AF151C01BF152C01CF1B9
:1017C00012004EC01DF14FC01EF150C01FF151C09C
:1017D00020F152C021F112004EC022F14FC023F17E
:1017E00050C024F151C025F152C026F112004EC064
:1017F00027F14FC028F150C029F151C02AF152C041
:101800002BF112002FC039F030C03AF031C03BF05C
:1018100032C03CF033C03DF012002FC03EF030C06B
:101820003FF031C040F032C041F033C042F012000E
:1018300039C02FF03AC030F03BC031F03CC032F03C
:101840003DC033F012003E363F3640364136423618
:10185000120039363A363B363C363D3612004232BB
:10186000413240323F323E3212003D323C323B3256
:101870003A323932120006D83436353636363736F3
:10188000383612002F3630363136323633361200C3
:10189000383237323632353234321200F9DF3332F1
:1018A0003232313230322F32120039AE04D03A683F
:1018B0003B683C683D6812003AAE03D03B683C6828
:1018C0003D6812003BAE02D03C683D6812003CAE61
:1018D00001D03D6812005C925BBE5C828CDE280EFB
:1018E0002C6ED89035EC0CF04FEC0CF003D82C2E6D
:1018F000F8D712004FEC16F00A0E2B6E00EE2FF008
:10190000EF50E8B6FD0FE8BED00FEE6E2B2EF8D7E5
:101910005CEC16F012003FD833AE09D0342AD8B4AC
:10192000352AD8B4362AD8B4372AD8B4382A02ECA3
:101930000BF035D030D833AE09D0342AD8B4352A9C
:10194000D8B4362AD8B4372AD8B4382A34C02FF0BD
:1019500035C030F036C031F037C032F038C033F027
:101960005BBE43EC13F0120016D834C02FF035C024
:1019700030F036C031F037C032F038C033F05BBEE3
:1019800043EC13F0120007D8FCEC0AF008D003D89F
:1019900002EC0BF004D0DEEC0EF0D3EF0CF090EC88
:1019A0000DF0F4EF0EF04CD803E1FBEC0AF01AD086
:1019B0001AD87F0E436E4350475E4450485A47C082
:1019C0002BF047520FE047BE06D0D8903BEC0CF00E
:1019D0002B2EFBD707D02B1E2B2AD8904EEC0CF0C9
:1019E0002B2EFBD712005B9E4DBE5B8E4D9EFBECFB
:1019F0000AF049C030F04AC031F04BC032F04CC060
:101A000033F04DC034F0D8903BEC0CF04FEC0CF0C0
:101A1000338E34C047F0346AD8903BEC0CF012009F
:101A2000040E2B6EEE6608D02B2EFCD7EECFE8FF0F
:101A30007F0B03E1D88401D0D8945CEC16F012003F
:101A40004FEC16F000EE49F0EBD74FEC16F000EE3D
:101A50004EF0E6D74FEC16F000EE53F0E1D74FEC26
:101A600016F000EE39F0DCD74FEC16F000EE3EF049
:101A7000D7D74FEC16F000EE2FF00A0E2B6EEE6665
:101A8000DBD72B2EFCD7D6D73D6A3CBE3D6835D080
:101A90003C6A3D6A3BAE31D03C683D682ED03B6A23
:101AA0003C6A3D6A3AAE29D03B683C683D6825D027
:101AB0003A6A3B6A3C6A3D6A39AE1FD03A683B6875
:101AC0003C683D681AD0FBEC0AF05B9E3D6A1DD075
:101AD000FBEC0AF05B9E3C6A3D6A17D0FBEC0AF017
:101AE0005B9E3B6A3C6A3D6A10D0FBEC0AF05B9E51
:101AF0003A6A3B6A3C6A3D6A08D0FBEC0AF05B9E9E
:101B00003DAE03D052EC13F05B8E39C034F03AC0D6
:101B100035F03BC036F03CC037F03DC038F000D067
:101B20007F0E476E000E486E39EC0DF006E1496AF3
:101B30004A6A4B6A4C6A4D6A36D0FAEC0DF007E0FF
:101B4000D8904EEC0CF0472AD8B4482AF6D734B0D7
:101B50000AD0D8903BEC0CF047064728D8B448068A
:101B6000D8B44752F4D730A00BD03080302AD8B444
:101B7000312AD8B4322AD8B4332AD8B4342ADDD79B
:101B80002F6A349047C034F04EEC0CF030C049F06E
:101B900031C04AF032C04BF033C04CF034C04DF08D
:101BA0004D9E5BBE4D8E1200496A4A6A4B6A4D6A71
:101BB000800E4C6EF5D749684A684B687F0E4C6EB4
:101BC0007F0E4D6EEDD77F0E396E000E3A6E485087
:101BD0003A5C02E14750395CD8B003D0ECDFD884DE
:101BE00001D0D894120048AE03D0DEDFD88401D0F3
:101BF000D89412004FEC16F000EE38F0040E2B6E65
:101C0000ED660AD02B2EFCD7010EEF6201D002D078
:101C1000EF6602D0D88401D0D8945CEC16F01200A4
:101C20003EC000F13FC001F140C002F141C003F1EC
:101C300042C004F15AEC0EF02FC007F130C008F199
:101C400031C009F132C00AF133C00BF100C139F0E3
:101C500001C13AF002C13BF003C13CF004C13DF0C8
:101C600040EC0EF007C134F008C135F009C136F080
:101C70000AC137F00BC138F05B9E5CB25B8E12007C
:101C8000BADC280E2C6ED89005D842EC0CF02C2E25
:101C9000FAD712004FEC16F0050E2B6E00EE39F05D
:101CA000D890EF50E8200700EE6E2B2EFAD75CECB0
:101CB00016F012004FEC16F09EDC280E2C6ED89019
:101CC00035EC0CF04FEC0CF000EE39F0050E2B6EFD
:101CD000EFAE02D0300EEF5EEFA602D0030EEF5E45
:101CE000EE522B2EF5D72C2EEAD75CEC16F0120014
:101CF00002D802EF0CF04FEC16F09ADD00EE2FF058
:101D000010EE3EF0040E2B6EE650EE5EE650EE5AFC
:101D10002B2EFCD75CEC16F0120002D802EF0CF070
:101D20004FEC16F085DD00EE2FF010EE3EF0E650A1
:101D3000EE26040E2B6EE650EE222B2EFCD75CEC2A
:101D400016F0120000C139F001C13AF002C13BF0B7
:101D500003C13CF004C13DF005C143F006C144F0AD
:101D6000120007C13EF008C13FF009C140F00AC1AE
:101D700041F00BC142F00CC145F00DC146F012001C
:101D800030C000F131C001F132C002F133C003F1C3
:101D900034C004F147C005F148C006F1120030C05C
:101DA00007F131C008F132C009F133C00AF134C083
:101DB0000BF147C00CF148C00DF112004EC049F0C4
:101DC0004FC04AF050C04BF051C04CF052C04DF0E3
:101DD000120053C049F054C04AF055C04BF056C0F1
:101DE0004CF057C04DF0120049C04EF04AC04FF0C1
:101DF0004BC050F04CC051F04DC052F0120049C0E1
:101E000053F04AC054F04BC055F04CC056F04DC092
:101E100057F012006CEC16F016E269EC16F013E2C3
:101E200025EC0DF01AE02AEC0DF017E081EC16F02D
:101E300004E325EC0DF001E306D084EC16F006E394
:101E40002AEC0DF003E3A9EC16F0120081EC16F079
:101E500003E39EEC16F003D00DD015EC0BF052BE50
:101E600003D057AE01D0528E52AE03D057BE01D030
:101E7000528E12001DD85B9E5BBA5B7E5BBC5B7EA4
:101E8000FFEC12F033C000F134C001F135C002F1B3
:101E900036C003F137C004F11ED890EC0EF002EC0E
:101EA0000CF00FEC0BF07F0E3E6E7BEC0EF01ED0B4
:101EB0005B9A5B9C52BE5B8A57BE5B8C7FDFF3EC08
:101EC0000CF05EDF86DFF3EC0CF069DFFAEC0AF071
:101ED00039DFB1EF0EF0FAEC0AF043C039F044C03C
:101EE0003AF045C03EF046C03FF012002FC047F028
:101EF00030C048F0FBEC0AF000C130F001C131F015
:101F000002C132F003C133F004C134F094EC0DF09F
:101F1000F4EF0EF06CEC16F009E269EC16F006E254
:101F200025EC0DF006E12AEC0DF019E1A9EC16F014
:101F3000120084EC16F003E381EC16F0F7E22AECD1
:101F40000DF010E19EEC16F052BE03D057AE01D05A
:101F5000528E52AE03D057BE01D0528E1200B3EC57
:101F600016F0F2D7A5DF5B9E5BBA5B7E5BBC5B7E47
:101F7000CDEC13F005DFAFDF7BEC0EF002EC0CF0E4
:101F80000FEC0BF07F0E3E6E90EC0EF0AFD72AEC0C
:101F90000DF001E11200577E00D06CEC16F004E267
:101FA00069EC16F001E203D0A9EC16F012002AEC5D
:101FB0000DF001E1120025EC0DF003E131EC0BF026
:101FC000120017D890EC0EF043C047F044C048F020
:101FD0005B9E33AE03D05B8E43EC13F02FC000F159
:101FE00030C001F131C002F132C003F133C004F15D
:101FF00081D75EDFFE0E476E000E486E4650445C91
:1020000002E14550435C27E013E3452AD8B4462A51
:102010004850465C02E14750455C07E10FEC0BF08D
:1020200043C045F044C046F016D0D89018DCE6D73F
:10203000432AD8B4442A4850445C02E14750435CE8
:1020400007E108EC0BF045C043F046C044F003D074
:10205000D8900BDCD3D75BBA52EC13F05BBC61ECCD
:1020600013F012003CEC0BF00AEF0FF025EC0DF032
:102070002DE052BE2CD06CEC16F028E247EC0BF0B1
:10208000ECD848DFCBEC0BF01E0E2E6E2E4E1ED081
:1020900026EC0BF05DEC0BF03DDF5DEC0BF07DDF33
:1020A000DCD838DF5DEC0BF05750525C0BE156503A
:1020B000515C08E15550505C05E154504F5C02E121
:1020C00053504E5C03E0CBEC0BF0E0D71200A9ECD0
:1020D00016F0120025EC0DF008E13F0E526E800E56
:1020E000516E4E6A4F6A506A120001013F0E266F10
:1020F000800E256F226B236B246B3F0E216F800EA9
:10210000206F1D6B1E6B1F6B0001D6EC0BF0CBEC30
:102110000BF022C10EF123C10FF124C110F125C132
:1021200011F126C112F11E0E2E6E52EC0BF089EC4D
:102130000BF0F0DE1BEC0BF0CDEC0FF01BEC0BF01A
:102140005750525C0BE15650515C08E15550505CC1
:1021500005E154504F5C02E153504E5C17E02E4EA7
:1021600015D047EC0BF094EC0BF06FD816DFECECCD
:102170000BF089EC0BF04EDEE1EC0BF068EC0BF0B1
:102180005DEC0BF047DECBEC0BF0CFD7120025EC6B
:102190000DF008E13F0E526E800E516E4E6A4F6A8E
:1021A000506A12004EC02CF14FC02DF150C02EF1DC
:1021B00051C02FF152C030F1C3EC0CF03BD82ADEF5
:1021C00089DFF7EC0BF02CC14EF02DC14FF02EC182
:1021D00050F02FC151F030C152F0CBEC0CF05B94B9
:1021E0005BBE5B8434C02EF027C14EF028C14FF097
:1021F00029C150F02AC151F02BC152F02E5206E0F5
:102200005BA4C5D85BB4D5D82E2EFAD71200420EE7
:10221000576E480E566E536A546A556A1200400E45
:10222000576E490E566E0F0E556EDA0E546EA20E94
:10223000536E1200400E576E130E566E5D0E556EA5
:102240008D0E546EDE0E536E12003F0E576E800ED2
:10225000566E536A546A556A1200400E576E536A9E
:10226000546A556A566A1200410E576E200E566E19
:10227000536A546A556A1200420E576EC80E566E63
:10228000536A546A556A1200440E576E7A0E566E9F
:10229000536A546A556A1200460E576E1C0E566EEB
:1022A000400E556E536A546A1200470E576EC30EA5
:1022B000566E500E556E536A546A1200490E576E90
:1022C000740E566E240E556E536A546A12004B0EED
:1022D000576E180E566E960E556E800E546E536ADB
:1022E00012004C0E576EBE0E566EBC0E556E200E72
:1022F000546E536A12004E0E576E6E0E566E6B0E73
:10230000556E280E546E536A12003D0E576ECC0E59
:10231000566ECC0E556ECC0E546ECD0E536E120012
:102320003C0E576E230E566ED70E556E0A0E546E27
:102330003D0E536E12003A0E576E830E566E120EFD
:10234000556E6E0E546E980E536E1200350E576E0B
:10235000860E566E370E556EBD0E546E060E536EBB
:102360001200300E576E890E566E700E556E5F0E4F
:10237000546E410E536E12002B0E576E8C0E566E1D
:10238000BC0E556ECC0E546E090E536E12006CDFEF
:102390000AEF0FF071DF0AEF0FF076DF0AEF0FF0B0
:1023A0007BDF0AEF0FF081DF0AEF0FF087DF0AEF24
:1023B0000FF05ADF8AEF0FF05FDF8AEF0FF064DF74
:1023C0008AEF0FF069DF8AEF0FF06FDF8AEF0FF00F
:1023D00075DF8AEF0FF025EC0DF003E1A9EC16F0A4
:1023E000120047EC0BF001013F0E176F800E166FC5
:1023F000136B146B156B000128DFC7EC0FF0D6ECE4
:102400000BF026EC0BF021DFCDEC0FF0E1EC0BF044
:1024100068EC0BF089EC0BF08AEC0FF0D6EC0BF0CB
:10242000ECEC0BF047EC0BF0280E2E6E52EC0BF0A0
:1024300014DFCDEC0FF0CBEC0BF068EC0BF09FEC65
:102440000BF00AEC0FF09FEC0BF00AEC0FF0D6EC5F
:102450000BF05DEC0BF08AEC0FF01BEC0BF0CDEC0D
:102460000FF01BEC0BF05750525C0BE15650515CD7
:1024700008E15550505C05E154504F5C02E1535067
:102480004E5C05E02E4E03D047EC0BF0CFD7E5DED7
:102490000AEF0FF00101276B000134EC11F048D86E
:1024A00006E3D9EC11F00101272B0001F6D793DFE9
:1024B000C1DE8AEC0FF0FAEC0AF027C134F0345296
:1024C00006E090EC0DF0FFEC0EF0CDEC0FF01200FA
:1024D0007ED83DAE14D042AE29D05AD83D50425C91
:1024E0000BE13C50415C08E13B50405C05E13A5057
:1024F0003F5C02E139503E5CD8B016D017D03DBEEB
:1025000002D042BE11D044D83D50425C0BE13C5059
:10251000415C08E13B50405C05E13A503F5C02E120
:1025200039503E5CD8B002D0D89001D0D88012008B
:102530004ED83DAE14D042AE29D02AD83D50425C90
:102540000BE13C50415C08E13B50405C05E13A50F6
:102550003F5C02E139503E5CD8B016D017D03DBE8A
:1025600002D042BE11D014D83D50425C0BE13C5029
:10257000415C08E13B50405C05E13A503F5C02E1C0
:1025800039503E5CD8B002D0D88001D0D89012002B
:1025900025EC0DF003E108EC0BF00FD0D89029ECFE
:1025A0000CF0D8903C323B323A3239323C8E2AEC35
:1025B0000DF003E10FEC0BF009D0D89023EC0CF0F8
:1025C000D890413240323F323E32418E12004EC0EE
:1025D00039F04FC03AF050C03BF051C03CF052C00F
:1025E0003DF053C03EF054C03FF055C040F056C0DF
:1025F00041F057C042F0120002D802EF0CF04FEC4D
:1026000016F037D8050E2B6E00EE3EF020EE2FF0C0
:10261000FBEC0AF010EE39F0050E2C6E2BC02DF0FD
:102620002C502D262D062D06EF50E602F350DE2607
:10263000D9CF58F0DACF59F0F450DE22E86ADE2222
:102640002D2EFCD758C0D9FF59C0DAFF2C2EE6D763
:10265000EE5220EE2FF0060E2D6E2B502D5EDE5228
:102660002D2EFDD72B2ED6D75CEC16F05BB20BD8F7
:1026700012005B923DAE02D015D85B7242AE02D022
:1026800020D85B7212002F1E301E311E321E331EE8
:102690002F2AD8B4302AD8B4312AD8B4322AD8B4A0
:1026A000332A1200391E3A1E3B1E3C1E3D1E392A9B
:1026B000D8B43A2AD8B43B2AD8B43C2AD8B43D2A54
:1026C00012003E1E3F1E401E411E421E3E2AD8B42E
:1026D0003F2AD8B4402AD8B4412AD8B4422A12009A
:1026E000C8DF4FEC16F0FBEC0AF0050E2B6E00EE87
:1026F0003EF0EE6605D02B2EFCD75CEC16F01200F7
:102700002B6A2B2AD89042BE1CD03E363F3640362C
:102710004136423642503D5C0BE141503C5C08E1A1
:1027200040503B5C05E13F503A5C02E13E50395C71
:10273000E8E2FBEC0AF0D8904232413240323F32BC
:102740003E3242503D5C0BE141503C5C08E1405060
:102750003B5C05E13F503A5C02E13E50395C0AE3E4
:102760003E50395E3F503A5A40503B5A41503C5AD5
:1027700042503D5A42EC0CF02B2EDDD777DF39C0AA
:102780003EF03AC03FF03BC040F03CC041F03DC09D
:1027900042F002EC0CF05CEF16F0290E2B6EFBEC15
:1027A0000AF042503D5C0BE141503C5C08E1405076
:1027B0003B5C05E13F503A5C02E13E50395C0BE383
:1027C0003E50395E3F503A5A40503B5A41503C5A75
:1027D00042503D5AD8803BEC0CF0D89029EC0CF0DC
:1027E00042503D5C0BE141503C5C08E140503B5C99
:1027F00005E13F503A5C02E13E50395C0BE33E504C
:10280000395E3F503A5A40503B5A41503C5A425030
:102810003D5AD8802B2EDFD712004FEC16F05B927A
:102820003DAE02D03FDF5B82FBEC0AF0280E2B6E40
:102830000A0E2C6E00EE2FF0EF500F0B2D6E050ED2
:102840002D5CD8A002D0030EEF26EF50F00B2D6EBA
:10285000500E2D5CD8A002D0300EEF26EC522C2E5C
:10286000EBD7D89029EC0CF03BEC0CF02B2EE0D7FA
:102870005CEC16F012006CEC16F015E284EC16F02D
:102880001CE22FD844D85AD85C941200030E586426
:1028900009D05966582A5BB4582A030E585E58501E
:1028A00038EC0AF01200F2DF000EF86E2D0EF76E13
:1028B000780EF66E30EC0AF01200E8DF000EF86ECB
:1028C0002D0EF76E7C0EF66E30EC0AF012006CECFA
:1028D00016F0E9E284EC16F0F0E203D82FD85C940D
:1028E00012004FEC16F000EE38F011EE31F00A0E47
:1028F0002D6EEDCF2BF02B382C6E56D82BC02CF034
:1029000053D82D2EF6D7E76A5CEC16F012004FEC88
:1029100016F0595210E001EE44F011EE44F0140E9E
:102920002B6E59C02CF0E5502B062C2EFCD7E5CF92
:10293000EDFF2B2EFCD75CEC16F012004FEC16F0DE
:102940000A0E2C6E59502C2658502C5CD8B002D050
:102950002CC058F05850595CD8A003D059C058F03A
:10296000582A5950585E5806090E2B6E58502B5E47
:1029700001EE31F02B5204E0EECFE8FF2B2EFCD716
:102980005BA405D02B0E5BBE2D0E13EC15F05B8007
:1029900019D85B9013D8595204E02C0E13EC15F0A3
:1029A00009D85CEC16F012002C500F0B3009E8CF60
:1029B000E6FF120059C02DF05C9606D0010E2D6E78
:1029C0005C9602D058C02DF02D5226E05BA006D0B8
:1029D000EFCF2BF0300E2B5CD8A45B905CA611D00F
:1029E0002DC039F0020E396202D00DEC15F0050E43
:1029F000396202D00DEC15F0080E396202D00DECF0
:102A000015F0EECFE8FF5BB003D013EC15F002D069
:102A10000FEC15F02D2EDAD71200200E04D0200E68
:102A20005CB4300E00D0296E5BA802D0010E5D6E42
:102A30005D6603D0295006EC0AF0010E5D6203D0FA
:102A4000295074EC09F012004FEC16F00A0E2B6EB0
:102A500059502B5E00EE2FF0EF502B4E0CD0EF5064
:102A60002B4E02D0EE52F8D7EE52396E490E396431
:102A700009D0010E06D00F0B396E040E396402D056
:102A8000100EEF260A0E2B6E00EE2FF0EF5007000F
:102A9000EE6EE86AEF222B2EF9D75CEC16F01200EE
:102AA0004FEC16F0050E2B6E0A0E2C6E00EE38F071
:102AB000EDCF39F03950F00B07E12C0639500F0BF0
:102AC00003E12C062B2EF4D72CC039F02C505CECF3
:102AD00016F01200B3EC16F0FBEC0AF00DEC14F05B
:102AE0002FC034F030C035F031C036F032C037F08E
:102AF00033C038F0050E586E596A5B945C945B984D
:102B00005C965D6A12006CEC16F045E284EC16F0FF
:102B100042E2DEEC0EF0D3EC0CF02FC000F130C03E
:102B200001F131C002F132C003F133C004F134C00D
:102B300039F035C03AF036C03BF037C03CF038C011
:102B40003DF00DEC14F02FC007F130C008F131C09A
:102B500009F132C00AF133C00BF100C139F001C1F3
:102B60003AF002C13BF003C13CF004C13DF06BEC14
:102B70000CF007C134F008C135F009C136F00AC1C4
:102B800037F00BC138F0140E586E0A0E596E5B9870
:102B90005C965C945D6A5B94120047EC0BF05A6A99
:102BA000529E25EC0DF014E034EC11F098EC12F08C
:102BB00001E004E3D9EC11F05A2AF6D725EC11F024
:102BC00068EC12F005E004E3C7EC11F05A06F6D702
:102BD00083EC15F026EC0BF052BE5B8E0B0E586E9C
:102BE0000A0E596E5B845B985D6A120067EC14F004
:102BF000650E13EC15F05B9E5ABE5B8E5ABE5A6C86
:102C000008EC0BF05AC039F06AEC15F05B8448DF31
:102C100039C058F067EC14F0120052EC0BF01BECCA
:102C20000BF0C7EC0FF0F7EC0BF07EEC0BF073EC55
:102C30000BF0C7EC0FF03CEC0BF027C14EF028C1B5
:102C40004FF029C150F02AC151F02BC152F08AEC4B
:102C50000FF0F7EC0BF094EC0BF073EC0BF0C7EC0F
:102C60000FF0B5EC0BF00AEC0FF01BEC0BF0CDEC19
:102C70000FF012004FEC16F008EC0BF0050E2B6E67
:102C800010EE2FF020EE39F0E6500F0BDF6EE63835
:102C9000F00BDE122B2EF8D75CEC16F01200E9CF09
:102CA00045F1EACF46F1E1CF47F1E2CF48F1D9CF84
:102CB00049F1DACF4AF1120045C1E9FF46C1EAFF06
:102CC00047C1E1FF48C1E2FF49C1D9FF4AC1DAFF6C
:102CD0001200E9EC0EF003D0DEEC0EF000D04D9EB9
:102CE0007F0E4D620CD0800E4C6207D04B6605D033
:102CF0004A6603D0496601D002D0D88001D0D8906E
:102D00001200E9EC0EF003D0DEEC0EF000D04D9E88
:102D10007F0E4D620BD0800E4C6208D04B6606D001
:102D20004A6604D0496602D0D88001D0D8901200FB
:102D300002D8F4EF0EF005D84D8E120002D8F4EF51
:102D40000EF07F0E4D6E800E4C6E496A4A6A4B6AD9
:102D5000120002D8F4EF0EF07F0E4D6E49684A68FB
:102D60004B684C68120002D8F4EF0EF0496A4A6AC8
:102D70004B6A4C6A4D6A12002D2D2D00494E4600BB
:020000040030CA
:0300010028193C7F
:020005003D803C
:0200000400F00A
:040000002D020000CD
:00000001FF
